 libimgegl

 Timestamp is 4be8cf49 (Tue May 11 12:30:17 2010)

 Preferred load address is 10000000

 Start         Length     Name                   Class
 0001:00000000 00000004H .CRT$XCA                CODE
 0001:00000004 00000004H .CRT$XCZ                CODE
 0001:00000008 00000004H .CRT$XIA                CODE
 0001:0000000c 00000004H .CRT$XIZ                CODE
 0001:00000010 00000004H .CRT$XPA                CODE
 0001:00000014 00000004H .CRT$XPZ                CODE
 0001:00000018 00000004H .CRT$XTA                CODE
 0001:0000001c 00000004H .CRT$XTZ                CODE
 0001:00000020 00001088H .rdata                  CODE
 0001:000010a8 00000026H .rdata$debug            CODE
 0001:000010d0 00008e14H .text                   CODE
 0001:00009ee4 00000018H .xdata                  CODE
 0001:00009efc 00000028H .idata$2                CODE
 0001:00009f24 00000014H .idata$3                CODE
 0001:00009f38 000000c8H .idata$4                CODE
 0001:0000a000 00000100H .idata$6                CODE
 0001:0000a100 00000541H .edata                  CODE
 0002:00000000 000000c8H .idata$5                DATA
 0002:000000c8 00000080H .data                   DATA
 0002:00000148 0000055cH .bss                    DATA
 0003:00000000 000003f0H .pdata                  DATA

  Address         Publics by Value              Rva+Base       Lib:Object

 0000:00000000       ___safe_se_handler_table   00000000     <absolute>
 0000:00000000       ___safe_se_handler_count   00000000     <absolute>
 0001:00000000       __xc_a                     10001000     corelib0:crt0init.obj
 0001:00000004       __xc_z                     10001004     corelib0:crt0init.obj
 0001:00000008       __xi_a                     10001008     corelib0:crt0init.obj
 0001:0000000c       __xi_z                     1000100c     corelib0:crt0init.obj
 0001:00000010       __xp_a                     10001010     corelib0:crt0init.obj
 0001:00000014       __xp_z                     10001014     corelib0:crt0init.obj
 0001:00000018       __xt_a                     10001018     corelib0:crt0init.obj
 0001:0000001c       __xt_z                     1000101c     corelib0:crt0init.obj
 0001:0000003c       ??_C@_0BD@BMHBHCAJ@eglDestroyImageKHR?$AA@ 1000103c     khronos_egl.obj
 0001:00000050       ??_C@_0BC@LFHEJBKG@eglCreateImageKHR?$AA@ 10001050     khronos_egl.obj
 0001:000000cc       aWSEGLPixelFormatBytesPerPixelShift 100010cc     khronos_egl.obj
 0001:000000f4       ??_C@_0BF@BLDJENPP@ExternalZBufferXSize?$AA@ 100010f4     khronos_egl.obj
 0001:0000010c       ??_C@_0BF@NAGFJOFK@ExternalZBufferYSize?$AA@ 1000110c     khronos_egl.obj
 0001:00000124       ??_C@_0N@DEBIAPND@WindowSystem?$AA@ 10001124     khronos_egl.obj
 0001:00000134       ??_C@_0BF@ENDLADNG@ForceExternalZBuffer?$AA@ 10001134     khronos_egl.obj
 0001:0000014c       ??_C@_0BC@OPBGHDMC@PDSFragBufferSize?$AA@ 1000114c     khronos_egl.obj
 0001:00000160       ??_C@_0BA@OONPEIO@ParamBufferSize?$AA@ 10001160     khronos_egl.obj
 0001:00000170       ??_C@_0BE@NCEPNDKE@ExternalZBufferMode?$AA@ 10001170     khronos_egl.obj
 0001:00000184       ??_C@_0BJ@FGEHHHOH@Imagination?5Technologies?$AA@ 10001184     khronos_egl.obj
 0001:000001a0       ??_C@_0M@CJFGPKFJ@1?44?5build?51?$AA@ 100011a0     khronos_egl.obj
 0001:000001b0       ??_C@_0KO@KNCFJIHN@EGL_KHR_image?5EGL_KHR_image_base@ 100011b0     khronos_egl.obj
 0001:00000260       ??_C@_0BC@KEPCFKB@OpenGL_ES?5OpenVG?5?$AA@ 10001260     khronos_egl.obj
 0001:000007b4       ??_C@_0P@MBENIONB@glMapBufferOES?$AA@ 100017b4     function_table.obj
 0001:000007c4       ??_C@_0BB@CEFEJGJJ@glUnmapBufferOES?$AA@ 100017c4     function_table.obj
 0001:000007d8       ??_C@_0BH@HANHAAH@glGetBufferPointervOES?$AA@ 100017d8     function_table.obj
 0001:000007f0       ??_C@_0BN@FPPCHDBA@glEGLImageTargetTexture2DOES?$AA@ 100017f0     function_table.obj
 0001:00000810       ??_C@_0CH@JLEJGINJ@glEGLImageTargetRenderbufferStor@ 10001810     function_table.obj
 0001:00000838       ??_C@_0BC@IBABPJFA@glMultiDrawArrays?$AA@ 10001838     function_table.obj
 0001:0000084c       ??_C@_0BE@MPDFJJLL@glMultiDrawElements?$AA@ 1000184c     function_table.obj
 0001:00000860       ??_C@_0BD@PIBFHNP@glTexBindStreamIMG?$AA@ 10001860     function_table.obj
 0001:00000874       ??_C@_0BM@MBNDOCOP@glGetTexStreamDeviceNameIMG?$AA@ 10001874     function_table.obj
 0001:00000890       ??_C@_0CD@OCNNIBKN@glGetTexStreamDeviceAttributeivI@ 10001890     function_table.obj
 0001:000008b4       ??_C@_0BB@JDDNIFAN@glGenProgramsARB?$AA@ 100018b4     function_table.obj
 0001:000008c8       ??_C@_0BE@EJCMOJPP@glDeleteProgramsARB?$AA@ 100018c8     function_table.obj
 0001:000008dc       ??_C@_0BB@OAGHGJAC@glBindProgramARB?$AA@ 100018dc     function_table.obj
 0001:000008f0       ??_C@_0BD@HIBLHAHB@glProgramStringARB?$AA@ 100018f0     function_table.obj
 0001:00000904       ??_C@_0BO@HGKLJN@glDisableVertexAttribArrayARB?$AA@ 10001904     function_table.obj
 0001:00000924       ??_C@_0BN@FKABDPBF@glEnableVertexAttribArrayARB?$AA@ 10001924     function_table.obj
 0001:00000944       ??_C@_0BJ@KNOILOPF@glVertexAttribPointerARB?$AA@ 10001944     function_table.obj
 0001:00000960       ??_C@_0BM@DIEJBCK@glProgramEnvParameter4xvIMG?$AA@ 10001960     function_table.obj
 0001:0000097c       ??_C@_0BL@IPGFFKBA@glProgramEnvParameter4xIMG?$AA@ 1000197c     function_table.obj
 0001:00000998       ??_C@_0BO@HBENEBND@glProgramLocalParameter4xvIMG?$AA@ 10001998     function_table.obj
 0001:000009b8       ??_C@_0BN@EBNCCGNG@glProgramLocalParameter4xIMG?$AA@ 100019b8     function_table.obj
 0001:000009d8       ??_C@_0BE@PEDBDIJA@glVertexAttrib4xIMG?$AA@ 100019d8     function_table.obj
 0001:000009ec       ??_C@_0BO@OHCIBKNP@glProgramLocalParameter4fvARB?$AA@ 100019ec     function_table.obj
 0001:00000a0c       ??_C@_0BN@DBLLDHNC@glProgramLocalParameter4fARB?$AA@ 10001a0c     function_table.obj
 0001:00000a2c       ??_C@_0BM@JFOBMKCG@glProgramEnvParameter4fvARB?$AA@ 10001a2c     function_table.obj
 0001:00000a48       ??_C@_0BL@PPAMELBE@glProgramEnvParameter4fARB?$AA@ 10001a48     function_table.obj
 0001:00000a64       ??_C@_0BE@IEFICJJE@glVertexAttrib4fARB?$AA@ 10001a64     function_table.obj
 0001:00000a78       ??_C@_0BE@BMGJDPBK@glGenerateMipmapOES?$AA@ 10001a78     function_table.obj
 0001:00000a8c       ??_C@_0CJ@FPBNJAAI@glGetFramebufferAttachmentParame@ 10001a8c     function_table.obj
 0001:00000ab8       ??_C@_0BN@CEGIKEBP@glFramebufferRenderbufferOES?$AA@ 10001ab8     function_table.obj
 0001:00000ad8       ??_C@_0BK@IBODAJKF@glFramebufferTexture2DOES?$AA@ 10001ad8     function_table.obj
 0001:00000af4       ??_C@_0BM@FKHNDAOE@glCheckFramebufferStatusOES?$AA@ 10001af4     function_table.obj
 0001:00000b10       ??_C@_0BF@GBILCPIM@glGenFramebuffersOES?$AA@ 10001b10     function_table.obj
 0001:00000b28       ??_C@_0BI@DJPGNLDO@glDeleteFramebuffersOES?$AA@ 10001b28     function_table.obj
 0001:00000b40       ??_C@_0BF@HIIGGHIK@glBindFramebufferOES?$AA@ 10001b40     function_table.obj
 0001:00000b58       ??_C@_0BD@PMGNFKPK@glIsFramebufferOES?$AA@ 10001b58     function_table.obj
 0001:00000b6c       ??_C@_0CA@ODMPPHIE@glGetRenderbufferParameterivOES?$AA@ 10001b6c     function_table.obj
 0001:00000b8c       ??_C@_0BJ@OLDCKGHK@glRenderbufferStorageOES?$AA@ 10001b8c     function_table.obj
 0001:00000ba8       ??_C@_0BG@EDIBBEEP@glGenRenderbuffersOES?$AA@ 10001ba8     function_table.obj
 0001:00000bc0       ??_C@_0BJ@GGLGLLBL@glDeleteRenderbuffersOES?$AA@ 10001bc0     function_table.obj
 0001:00000bdc       ??_C@_0BG@FPKCPFFN@glBindRenderbufferOES?$AA@ 10001bdc     function_table.obj
 0001:00000bf4       ??_C@_0BE@PCDGPFM@glIsRenderbufferOES?$AA@ 10001bf4     function_table.obj
 0001:00000c08       ??_C@_0O@BKAEAEDL@glGetTexGenxv?$AA@ 10001c08     function_table.obj
 0001:00000c18       ??_C@_0O@MLMIKEB@glGetTexGenfv?$AA@ 10001c18     function_table.obj
 0001:00000c28       ??_C@_0O@HOAMNHM@glGetTexGeniv?$AA@ 10001c28     function_table.obj
 0001:00000c38       ??_C@_0L@PFIPKMPO@glTexGenxv?$AA@ 10001c38     function_table.obj
 0001:00000c44       ??_C@_09DJAOHNFO@glTexGenx?$AA@ 10001c44     function_table.obj
 0001:00000c50       ??_C@_0L@ODDHCCIE@glTexGenfv?$AA@ 10001c50     function_table.obj
 0001:00000c5c       ??_C@_09ONEPECIB@glTexGenf?$AA@ 10001c5c     function_table.obj
 0001:00000c68       ??_C@_0L@OIGLGFLJ@glTexGeniv?$AA@ 10001c68     function_table.obj
 0001:00000c74       ??_C@_09GKNHFOEO@glTexGeni?$AA@ 10001c74     function_table.obj
 0001:00000c80       ??_C@_0BE@LLLCIIOO@glBlendFuncSeparate?$AA@ 10001c80     function_table.obj
 0001:00000c94       ??_C@_0BI@JNHDNJAG@glBlendEquationSeparate?$AA@ 10001c94     function_table.obj
 0001:00000cac       ??_C@_0BA@PFHILPAN@glBlendEquation?$AA@ 10001cac     function_table.obj
 0001:00000cbc       ??_C@_0BC@DEKNHIDE@glQueryMatrixxOES?$AA@ 10001cbc     function_table.obj
 0001:00000cd0       ??_C@_0P@LKNACIFH@glDrawTexxvOES?$AA@ 10001cd0     function_table.obj
 0001:00000ce0       ??_C@_0P@IDAMELLM@glDrawTexfvOES?$AA@ 10001ce0     function_table.obj
 0001:00000cf0       ??_C@_0P@HCFKPJGJ@glDrawTexivOES?$AA@ 10001cf0     function_table.obj
 0001:00000d00       ??_C@_0P@NABHNIJE@glDrawTexsvOES?$AA@ 10001d00     function_table.obj
 0001:00000d10       ??_C@_0O@GOFANFJA@glDrawTexxOES?$AA@ 10001d10     function_table.obj
 0001:00000d20       ??_C@_0O@LBIAPMHD@glDrawTexfOES?$AA@ 10001d20     function_table.obj
 0001:00000d30       ??_C@_0O@DDNAGLKC@glDrawTexiOES?$AA@ 10001d30     function_table.obj
 0001:00000d40       ??_C@_0O@BJIAOEIB@glDrawTexsOES?$AA@ 10001d40     function_table.obj
 0001:00000d50       ??_C@_0BD@PCEFFFDF@glWeightPointerOES?$AA@ 10001d50     function_table.obj
 0001:00000d64       ??_C@_0BI@BEEEECPN@glMatrixIndexPointerOES?$AA@ 10001d64     function_table.obj
 0001:00000d7c       ??_C@_0CE@HEFPEHID@glLoadPaletteFromModelViewMatrix@ 10001d7c     function_table.obj
 0001:00000da0       ??_C@_0BK@NDELAMFO@glCurrentPaletteMatrixOES?$AA@ 10001da0     function_table.obj
 0001:00000dbc       ??_C@_0BG@PIPFALFL@glPointSizePointerOES?$AA@ 10001dbc     function_table.obj
 0001:00000dd4       ??_C@_0BD@PEKIFPFH@glProgramBinaryOES?$AA@ 10001dd4     function_table.obj
 0001:00000de8       ??_C@_0BG@GMFJDPBI@glGetProgramBinaryOES?$AA@ 10001de8     function_table.obj
 0001:00000e00       ??_C@_0BK@MJMMJBHE@vgCreateEGLImageTargetKHR?$AA@ 10001e00     function_table.obj
 0001:00000e1c       ??_C@_0BO@GEMPEOEK@WSEGL_GetFunctionTablePointer?$AA@ 10001e1c     generic_ws.obj
 0001:00000e3c       ??_C@_0L@FNOAAMKB@nullws?4dll?$AA@ 10001e3c     generic_ws.obj
 0001:00000e48       ??_C@_09CKNCACDD@wsegl?4dll?$AA@ 10001e48     generic_ws.obj
 0001:00000e54       ??_C@_0M@OPOBFDCB@glGetString?$AA@ 10001e54     generic_ws.obj
 0001:00000e60       ??_C@_0P@MADFBLIB@libGLES_CM?4dll?$AA@ 10001e60     generic_ws.obj
 0001:00000e70       ??_C@_0O@HFAAEHFL@libGLESv2?4dll?$AA@ 10001e70     generic_ws.obj
 0001:00000e80       ??_C@_0M@FLHNHFPG@vgGetString?$AA@ 10001e80     generic_ws.obj
 0001:00000e8c       ??_C@_0O@LFGHKFEJ@libOpenVG?4dll?$AA@ 10001e8c     generic_ws.obj
 0001:00000ea0       SRV_pixel_format_alpha     10001ea0     srv.obj
 0001:00000f08       SRV_pixel_format_red       10001f08     srv.obj
 0001:00000f70       SRV_pixel_format_green     10001f70     srv.obj
 0001:00000fd8       SRV_pixel_format_blue      10001fd8     srv.obj
 0001:00001040       SRV_pixel_format_width     10002040     srv.obj
 0001:000010d0       EGLThreadLock              100020d0 f   khronos_egl.obj
 0001:000010dc       EGLThreadUnlock            100020dc f   khronos_egl.obj
 0001:00001114       _TlsInit                   10002114 f   khronos_egl.obj
 0001:00001440       GetKEGLDisplay             10002440 f   khronos_egl.obj
 0001:00001494       IsEGLContext               10002494 f   khronos_egl.obj
 0001:000019d8       KEGLSurfaceUnbind          100029d8 f   khronos_egl.obj
 0001:00001a38       KEGLSurfaceBind            10002a38 f   khronos_egl.obj
 0001:00001a48       IMGeglGetError             10002a48 f   khronos_egl.obj
 0001:00001a68       IMGeglGetDisplay           10002a68 f   khronos_egl.obj
 0001:00001b70       IMGeglInitialize           10002b70 f   khronos_egl.obj
 0001:00001e20       IMGeglTerminate            10002e20 f   khronos_egl.obj
 0001:000020f8       IMGeglQueryString          100030f8 f   khronos_egl.obj
 0001:000021e0       IMGeglGetProcAddress       100031e0 f   khronos_egl.obj
 0001:00002410       IMGeglGetConfigs           10003410 f   khronos_egl.obj
 0001:000024ec       IMGeglChooseConfig         100034ec f   khronos_egl.obj
 0001:00002768       IMGeglGetConfigAttrib      10003768 f   khronos_egl.obj
 0001:00002854       IMGeglCreateWindowSurface  10003854 f   khronos_egl.obj
 0001:00002c94       IMGeglCreatePixmapSurface  10003c94 f   khronos_egl.obj
 0001:000030c4       IMGeglCreatePbufferSurface 100040c4 f   khronos_egl.obj
 0001:00003730       IMGeglDestroySurface       10004730 f   khronos_egl.obj
 0001:00003818       IMGeglQuerySurface         10004818 f   khronos_egl.obj
 0001:00003b68       IMGeglCreateContext        10004b68 f   khronos_egl.obj
 0001:00003f74       IMGeglDestroyContext       10004f74 f   khronos_egl.obj
 0001:00004044       IMGeglMakeCurrent          10005044 f   khronos_egl.obj
 0001:0000461c       IMGeglGetCurrentContext    1000561c f   khronos_egl.obj
 0001:0000464c       IMGeglGetCurrentSurface    1000564c f   khronos_egl.obj
 0001:000046bc       IMGeglGetCurrentDisplay    100056bc f   khronos_egl.obj
 0001:00004700       IMGeglQueryContext         10005700 f   khronos_egl.obj
 0001:000048f8       IMGeglWaitGL               100058f8 f   khronos_egl.obj
 0001:000049b8       IMGeglWaitNative           100059b8 f   khronos_egl.obj
 0001:00004ab8       IMGeglSwapBuffers          10005ab8 f   khronos_egl.obj
 0001:00004cb8       IMGeglCopyBuffers          10005cb8 f   khronos_egl.obj
 0001:00004f5c       IMGeglSwapInterval         10005f5c f   khronos_egl.obj
 0001:0000509c       IMGeglSurfaceAttrib        1000609c f   khronos_egl.obj
 0001:00005240       IMGeglBindTexImage         10006240 f   khronos_egl.obj
 0001:00005460       IMGeglReleaseTexImage      10006460 f   khronos_egl.obj
 0001:0000559c       IMGeglCreatePbufferFromClientBuffer 1000659c f   khronos_egl.obj
 0001:00005a60       IMGeglBindAPI              10006a60 f   khronos_egl.obj
 0001:00005ad0       IMGeglQueryAPI             10006ad0 f   khronos_egl.obj
 0001:00005b28       IMGeglWaitClient           10006b28 f   khronos_egl.obj
 0001:00005c64       IMGeglReleaseThread        10006c64 f   khronos_egl.obj
 0001:00005ccc       KEGLRecreateDrawable       10006ccc f   khronos_egl.obj
 0001:00005f84       KEGLBindImage              10006f84 f   egl_eglimage.obj
 0001:00005f94       KEGLUnbindImage            10006f94 f   egl_eglimage.obj
 0001:00005f98       KEGLGetImageSource         10006f98 f   egl_eglimage.obj
 0001:00006014       IMGeglCreateImageKHR       10007014 f   egl_eglimage.obj
 0001:0000647c       IMGeglDestroyImageKHR      1000747c f   egl_eglimage.obj
 0001:00006520       TerminateImages            10007520 f   egl_eglimage.obj
 0001:0000656c       CFG_Variants               1000756c f   cfg.obj
 0001:00006884       CFG_GenerateVariant        10007884 f   cfg.obj
 0001:00006ae8       CFG_Match                  10007ae8 f   cfg.obj
 0001:00006b84       CFG_PrepareConfigFilter    10007b84 f   cfg.obj
 0001:00006d64       CFG_CompatibleConfigs      10007d64 f   cfg.obj
 0001:00006dc0       CFG_Compare                10007dc0 f   cfg.obj
 0001:00006fcc       CFGC_CreateAvArray         10007fcc f   cfg_core.obj
 0001:00007008       CFGC_CopyNl                10008008 f   cfg_core.obj
 0001:00007040       CFGC_Unlink                10008040 f   cfg_core.obj
 0001:00007084       CFGC_SetAttrib             10008084 f   cfg_core.obj
 0001:000070f8       CFGC_GetAttrib             100080f8 f   cfg_core.obj
 0001:0000717c       CFGC_GetAttribNoAccumulate 1000817c f   cfg_core.obj
 0001:000071cc       CFGC_ModifyAvArrayNl       100081cc f   cfg_core.obj
 0001:00007f34       IMGGetDummyFunction        10008f34 f   function_table.obj
 0001:0000801c       IMGFindLibraryToLoad       1000901c f   function_table.obj
 0001:00008160       LoadWSModule               10009160 f   generic_ws.obj
 0001:00008260       UnloadModule               10009260 f   generic_ws.obj
 0001:00008278       LoadOGLES1AndGetFunctions  10009278 f   generic_ws.obj
 0001:00008314       LoadOGLES2AndGetFunctions  10009314 f   generic_ws.obj
 0001:000083b0       LoadOVGAndGetFunctions     100093b0 f   generic_ws.obj
 0001:0000844c       KEGLGetDrawableParameters  1000944c f   generic_ws.obj
 0001:0000878c       GWS_CreatePBufferDrawable  1000978c f   generic_ws.obj
 0001:00008840       GWS_DeletePBufferDrawable  10009840 f   generic_ws.obj
 0001:00008864       ENV_CreateGlobalData       10009864 f   egl_win32.obj
 0001:00008880       ENV_DestroyGlobalData      10009880 f   egl_win32.obj
 0001:000088a4       ENV_GetGlobalData          100098a4 f   egl_win32.obj
 0001:00008a28       PVR_qsort_s                10009a28 f   qsort_s.obj
 0001:00008a4c       SRV_FindPVRPixelFormat     10009a4c f   srv.obj
 0001:00008af4       SRV_ServicesInit           10009af4 f   srv.obj
 0001:00008af8       SRV_ServicesDeInit         10009af8 f   srv.obj
 0001:00008afc       KEGLCreateRenderSurface    10009afc f   srv.obj
 0001:00008b20       KEGLDestroyRenderSurface   10009b20 f   srv.obj
 0001:00008b24       KEGLResizeRenderSurface    10009b24 f   srv.obj
 0001:00008b40       SRV_CreateSurface          10009b40 f   srv.obj
 0001:00008c74       SRV_DestroySurface         10009c74 f   srv.obj
 0001:00008c7c       SRV_SGXServicesInit        10009c7c f   srv_sgx.obj
 0001:00008e74       SRV_SGXServicesDeInit      10009e74 f   srv_sgx.obj
 0001:00008fc4       KEGL_SGXCreateRenderSurface 10009fc4 f   srv_sgx.obj
 0001:00009344       KEGL_SGXDestroyRenderSurface 1000a344 f   srv_sgx.obj
 0001:0000945c       KEGL_SGXResizeRenderSurface 1000a45c f   srv_sgx.obj
 0001:00009694       SGXAllocatePBufferDeviceMem 1000a694 f   srv_sgx.obj
 0001:00009704       KEGL_SGXSetContextPriority 1000a704 f   srv_sgx.obj
 0001:00009728       TLS_Open                   1000a728 f   tls.obj
 0001:00009788       TLS_Close                  1000a788 f   tls.obj
 0001:000097bc       IMGEGL_GetTLSID            1000a7bc f   wince6_tls.obj
 0001:000097c4       IMGEGL_GetTLSValue         1000a7c4 f   wince6_tls.obj
 0001:000097f4       IMGEGL_SetTLSValue         1000a7f4 f   wince6_tls.obj
 0001:00009838       PVRSRVLockMutex            1000a838 f   srvclum:SRVCLUM.dll
 0001:00009848       PVRSRVUnlockMutex          1000a848 f   srvclum:SRVCLUM.dll
 0001:00009858       PVRSRVDestroyMutex         1000a858 f   srvclum:SRVCLUM.dll
 0001:00009868       PVRSRVCreateMutex          1000a868 f   srvclum:SRVCLUM.dll
 0001:00009878       PVRSRVFreeAppHintState     1000a878 f   srvclum:SRVCLUM.dll
 0001:00009888       PVRSRVGetAppHint           1000a888 f   srvclum:SRVCLUM.dll
 0001:00009898       PVRSRVCreateAppHintState   1000a898 f   srvclum:SRVCLUM.dll
 0001:000098a8       PVRSRVFreeDeviceMem        1000a8a8 f   srvclum:SRVCLUM.dll
 0001:000098b8       PVRSRVUnloadLibrary        1000a8b8 f   srvclum:SRVCLUM.dll
 0001:000098c8       PVRSRVGetLibFuncAddr       1000a8c8 f   srvclum:SRVCLUM.dll
 0001:000098d8       PVRSRVLoadLibrary          1000a8d8 f   srvclum:SRVCLUM.dll
 0001:000098e8       PVRSRVMemCopy              1000a8e8 f   srvclum:SRVCLUM.dll
 0001:000098f8       SGXCreateTransferContext   1000a8f8 f   srvclum:SRVCLUM.dll
 0001:00009908       SGXCreateRenderContext     1000a908 f   srvclum:SRVCLUM.dll
 0001:00009918       PVRSRVGetMiscInfo          1000a918 f   srvclum:SRVCLUM.dll
 0001:00009928       SGXGetClientInfo           1000a928 f   srvclum:SRVCLUM.dll
 0001:00009938       PVRSRVCreateDeviceMemContext 1000a938 f   srvclum:SRVCLUM.dll
 0001:00009948       PVRSRVAcquireDeviceData    1000a948 f   srvclum:SRVCLUM.dll
 0001:00009958       PVRSRVEnumerateDevices     1000a958 f   srvclum:SRVCLUM.dll
 0001:00009968       PVRSRVConnect              1000a968 f   srvclum:SRVCLUM.dll
 0001:00009978       PVRSRVDisconnect           1000a978 f   srvclum:SRVCLUM.dll
 0001:00009988       PVRSRVDestroyDeviceMemContext 1000a988 f   srvclum:SRVCLUM.dll
 0001:00009998       SGXReleaseClientInfo       1000a998 f   srvclum:SRVCLUM.dll
 0001:000099a8       PVRSRVReleaseMiscInfo      1000a9a8 f   srvclum:SRVCLUM.dll
 0001:000099b8       SGXDestroyRenderContext    1000a9b8 f   srvclum:SRVCLUM.dll
 0001:000099c8       SGXDestroyTransferContext  1000a9c8 f   srvclum:SRVCLUM.dll
 0001:000099d8       PVRSRVAllocDeviceMem       1000a9d8 f   srvclum:SRVCLUM.dll
 0001:000099e8       SGXRemoveRenderTarget      1000a9e8 f   srvclum:SRVCLUM.dll
 0001:000099f8       SGXAddRenderTarget         1000a9f8 f   srvclum:SRVCLUM.dll
 0001:00009a08       PVRSRVReleaseThreadQuanta  1000aa08 f   srvclum:SRVCLUM.dll
 0001:00009a18       SGXSetContextPriority      1000aa18 f   srvclum:SRVCLUM.dll
 0001:00009a28       __GetUserKData             1000aa28 f   coredll:COREDLL.dll
 0001:00009a38       TlsCall                    1000aa38 f   coredll:COREDLL.dll
 0001:00009a48       TlsGetValue                1000aa48 f   coredll:COREDLL.dll
 0001:00009a58       TlsSetValue                1000aa58 f   coredll:COREDLL.dll
 0001:00009a68       DllMain                    1000aa68 f   corelib0:dllmain.obj
 0001:00009b84       _DllMainCRTStartup         1000ab84 f   corelib0:pegdmain.obj
 0001:00009bb4       __GSHandlerCheckCommon     1000abb4 f   corelib0:gshandler.obj
 0001:00009bf0       __GSHandlerCheck           1000abf0 f   corelib0:gshandler.obj
 0001:00009c14       __security_init_cookie     1000ac14 f   corelib0:seccinit.obj
 0001:00009c70       __security_check_cookie    1000ac70 f   corelib0:armsecgs.obj
 0001:00009c84       __gsfailure                1000ac84 f   corelib0:armsecgs.obj
 0001:00009d90       _cexit                     1000ad90 f   corelib0:cexit.obj
 0001:00009dac       _initterm                  1000adac f   corelib0:crt0dat.obj
 0001:00009de0       _cinit                     1000ade0 f   corelib0:crt0dat.obj
 0001:00009e14       strcpy                     1000ae14 f   corelib1:COREDLL.dll
 0001:00009e24       free                       1000ae24 f   corelib1:COREDLL.dll
 0001:00009e34       strncmp                    1000ae34 f   corelib1:COREDLL.dll
 0001:00009e44       strlen                     1000ae44 f   corelib1:COREDLL.dll
 0001:00009e54       calloc                     1000ae54 f   corelib1:COREDLL.dll
 0001:00009e64       realloc                    1000ae64 f   corelib1:COREDLL.dll
 0001:00009e74       strcmp                     1000ae74 f   corelib1:COREDLL.dll
 0001:00009e84       _XcptFilter                1000ae84 f   corelib1:COREDLL.dll
 0001:00009e94       __C_specific_handler       1000ae94 f   corelib1:COREDLL.dll
 0001:00009ea4       __security_gen_cookie2     1000aea4 f   corelib1:COREDLL.dll
 0001:00009eb4       __report_gsfailure         1000aeb4 f   corelib1:COREDLL.dll
 0001:00009ec4       DisableThreadLibraryCalls  1000aec4 f   coredll:COREDLL.dll
 0001:00009ed4       TerminateProcess           1000aed4 f   coredll:COREDLL.dll
 0001:00009efc       __IMPORT_DESCRIPTOR_SRVCLUM 1000aefc     srvclum:SRVCLUM.dll
 0001:00009f10       __IMPORT_DESCRIPTOR_COREDLL 1000af10     coredll:COREDLL.dll
 0001:00009f24       __NULL_IMPORT_DESCRIPTOR   1000af24     srvclum:SRVCLUM.dll
 0002:00000000       __imp_TerminateProcess     1000c000     coredll:COREDLL.dll
 0002:00000004       __imp___report_gsfailure   1000c004     corelib1:COREDLL.dll
 0002:00000008       __imp___security_gen_cookie2 1000c008     corelib1:COREDLL.dll
 0002:0000000c       __imp___C_specific_handler 1000c00c     corelib1:COREDLL.dll
 0002:00000010       __imp__XcptFilter          1000c010     corelib1:COREDLL.dll
 0002:00000014       __imp_strcmp               1000c014     corelib1:COREDLL.dll
 0002:00000018       __imp_realloc              1000c018     corelib1:COREDLL.dll
 0002:0000001c       __imp_calloc               1000c01c     corelib1:COREDLL.dll
 0002:00000020       __imp_strlen               1000c020     corelib1:COREDLL.dll
 0002:00000024       __imp_strncmp              1000c024     corelib1:COREDLL.dll
 0002:00000028       __imp_free                 1000c028     corelib1:COREDLL.dll
 0002:0000002c       __imp_strcpy               1000c02c     corelib1:COREDLL.dll
 0002:00000030       __imp_TlsSetValue          1000c030     coredll:COREDLL.dll
 0002:00000034       __imp_TlsGetValue          1000c034     coredll:COREDLL.dll
 0002:00000038       __imp_TlsCall              1000c038     coredll:COREDLL.dll
 0002:0000003c       __imp___GetUserKData       1000c03c     coredll:COREDLL.dll
 0002:00000040       __imp_DisableThreadLibraryCalls 1000c040     coredll:COREDLL.dll
 0002:00000044       \177COREDLL_NULL_THUNK_DATA 1000c044     coredll:COREDLL.dll
 0002:00000048       __imp_PVRSRVDisconnect     1000c048     srvclum:SRVCLUM.dll
 0002:0000004c       __imp_PVRSRVDestroyDeviceMemContext 1000c04c     srvclum:SRVCLUM.dll
 0002:00000050       __imp_SGXReleaseClientInfo 1000c050     srvclum:SRVCLUM.dll
 0002:00000054       __imp_PVRSRVReleaseMiscInfo 1000c054     srvclum:SRVCLUM.dll
 0002:00000058       __imp_SGXDestroyRenderContext 1000c058     srvclum:SRVCLUM.dll
 0002:0000005c       __imp_PVRSRVConnect        1000c05c     srvclum:SRVCLUM.dll
 0002:00000060       __imp_PVRSRVAllocDeviceMem 1000c060     srvclum:SRVCLUM.dll
 0002:00000064       __imp_SGXRemoveRenderTarget 1000c064     srvclum:SRVCLUM.dll
 0002:00000068       __imp_SGXAddRenderTarget   1000c068     srvclum:SRVCLUM.dll
 0002:0000006c       __imp_PVRSRVReleaseThreadQuanta 1000c06c     srvclum:SRVCLUM.dll
 0002:00000070       __imp_SGXSetContextPriority 1000c070     srvclum:SRVCLUM.dll
 0002:00000074       __imp_PVRSRVEnumerateDevices 1000c074     srvclum:SRVCLUM.dll
 0002:00000078       __imp_PVRSRVAcquireDeviceData 1000c078     srvclum:SRVCLUM.dll
 0002:0000007c       __imp_PVRSRVCreateDeviceMemContext 1000c07c     srvclum:SRVCLUM.dll
 0002:00000080       __imp_SGXGetClientInfo     1000c080     srvclum:SRVCLUM.dll
 0002:00000084       __imp_PVRSRVGetMiscInfo    1000c084     srvclum:SRVCLUM.dll
 0002:00000088       __imp_SGXCreateRenderContext 1000c088     srvclum:SRVCLUM.dll
 0002:0000008c       __imp_SGXCreateTransferContext 1000c08c     srvclum:SRVCLUM.dll
 0002:00000090       __imp_PVRSRVMemCopy        1000c090     srvclum:SRVCLUM.dll
 0002:00000094       __imp_PVRSRVLoadLibrary    1000c094     srvclum:SRVCLUM.dll
 0002:00000098       __imp_PVRSRVGetLibFuncAddr 1000c098     srvclum:SRVCLUM.dll
 0002:0000009c       __imp_PVRSRVUnloadLibrary  1000c09c     srvclum:SRVCLUM.dll
 0002:000000a0       __imp_PVRSRVFreeDeviceMem  1000c0a0     srvclum:SRVCLUM.dll
 0002:000000a4       __imp_PVRSRVCreateAppHintState 1000c0a4     srvclum:SRVCLUM.dll
 0002:000000a8       __imp_PVRSRVGetAppHint     1000c0a8     srvclum:SRVCLUM.dll
 0002:000000ac       __imp_PVRSRVFreeAppHintState 1000c0ac     srvclum:SRVCLUM.dll
 0002:000000b0       __imp_PVRSRVCreateMutex    1000c0b0     srvclum:SRVCLUM.dll
 0002:000000b4       __imp_PVRSRVDestroyMutex   1000c0b4     srvclum:SRVCLUM.dll
 0002:000000b8       __imp_PVRSRVUnlockMutex    1000c0b8     srvclum:SRVCLUM.dll
 0002:000000bc       __imp_SGXDestroyTransferContext 1000c0bc     srvclum:SRVCLUM.dll
 0002:000000c0       __imp_PVRSRVLockMutex      1000c0c0     srvclum:SRVCLUM.dll
 0002:000000c4       \177SRVCLUM_NULL_THUNK_DATA 1000c0c4     srvclum:SRVCLUM.dll
 0002:00000140       __security_cookie          1000c140     corelib0:seccinit.obj
 0002:00000144       __security_cookie_complement 1000c144     corelib0:seccinit.obj
 0002:00000694       _exitflag                  1000c694     corelib0:cexit.obj
 0002:00000698       __onexitend                1000c698     <common>
 0002:0000069c       __onexitbegin              1000c69c     <common>
 0002:000006a0       _pRawDllMain               1000c6a0     <common>

 entry point at        0001:00009b84

 Static symbols

 0001:000010e8       GlobalDataDeinit           100020e8 f   khronos_egl.obj
 0001:0000139c       _TlsDeInit                 1000239c f   khronos_egl.obj
 0001:000014c8       _InitialiseContextMode     100024c8 f   khronos_egl.obj
 0001:0000161c       _ContextDelete             1000261c f   khronos_egl.obj
 0001:00001728       _SurfaceDelete             10002728 f   khronos_egl.obj
 0001:00001818       _ValidateAttribList        10002818 f   khronos_egl.obj
 0001:00005ee4       UnbindImage                10006ee4 f   egl_eglimage.obj
 0001:00006580       DeriveCfg                  10007580 f   cfg.obj
 0001:00007228       DummyglMapBufferOES        10008228 f   function_table.obj
 0001:00007314       DummyglUnmapBufferOES      10008314 f   function_table.obj
 0001:000073f4       DummyglGetBufferPointervOES 100083f4 f   function_table.obj
 0001:000074e4       DummyglEGLImageTargetTexture2DOES 100084e4 f   function_table.obj
 0001:000075c8       DummyglEGLImageTargetRenderbufferStorageOES 100085c8 f   function_table.obj
 0001:000076ac       DummyglMultiDrawArrays     100086ac f   function_table.obj
 0001:000077a8       DummyglMultiDrawElements   100087a8 f   function_table.obj
 0001:000078c0       IMGSearchGLES1Extension    100088c0 f   function_table.obj
 0001:000088b4       _partition                 100098b4 f   qsort_s.obj
 0001:000089bc       _sort                      100099bc f   qsort_s.obj
 0001:00008f08       SetupTerminateBuffers      10009f08 f   srv_sgx.obj
 0001:00009a88       _DllMainCRTStartupHelper   1000aa88 f   corelib0:pegdmain.obj
 0001:00009cc8       doexit                     1000acc8 f   corelib0:cexit.obj
